S01100006B65726E656C2D726F6D2E6D6F7474
S325000000000020002001010000FF010000010200000302000005020000070200000000000080
S32500000020000000000000000000000000F50A000000000000000000002B0A0000850B0000F6
S32500000040FD010000FD010000FD010000FD010000FD010000FD010000FD010000FD010000AA
S32500000060FD010000FD010000FD010000FD010000FD010000FD010000FD010000FD0100008A
S32500000080FD010000FD010000FD010000FD010000FD010000FD010000FD010000FD0100006A
S325000000A0FD010000FD010000FD010000FD010000FD010000FD010000FD010000FD0100004A
S325000000C0FD010000FD010000FD010000FD010000FD010000FD010000FD010000FD0100002A
S325000000E0FD010000FD010000FD010000FD010000FD010000FD010000330B0000090A0000B5
S3250000010000F086F80C490D4A0D4BA3EB020301C901C2043B7FF4FBAF0A49084A0A600A4989
S325000001200A4A0B4B9B1A00F0058001C901C2043B7FF4FBAF00F00EB80000000000E0FF1F48
S3250000014000E1FF1F08ED00E07024000000E1FF1F30E1FF1F1A4A1B4B9B1A00F005800020EF
S3250000016001C2043B7FF4FCAF174DAA4288BF154616480560164D1748056000F0ADF9164D84
S325000001802E68164F3E4056F440762E60144D00262E60144D144E2E60144D2E68CCF2300601
S325000001A02E60134800F014FA124800F011FA124D2E6856F002062E6002F068F8FEE70000F5
S325000001C030E1FF1F2407002000E0FF1F34E1FF1F801D002030E1FF1F0CED00E0FFF8FFFFB4
S325000001E01CED00E020ED00E00000F0102CE400E02F0000002E00000014ED00E0FEE7FEE72B
S32500000200FEE7FEE7FEE7FEE7704700BF704700BF2DE9F00F4FF4E0514EF2515B41F6AE2AD4
S32500000220C4F2010141F208094FF010084FF0140CC1F6CC2BCEF2335AC1F800B00022C1F8C7
S3250000024000A0182701211C26C4F20109C4F20108C4F2010CC9F800202025C8F800202824C1
S32500000260CCF80010C4F201078121C4F20106396030203160C4F201058321C4F20104296069
S3250000028013462260C4F201005C220260C4F201031968042241F002011960C4F201021368A4
S325000002A09907FCD534200023C4F2010038210360C4F201013C2201200860C4F2010209215B
S325000002C011601C46C4F201031968042241F010011960C4F201021368DB06FCD50020C4F26D
S325000002E001000368042143F040030360C4F2010103680A6803F0E00302F0E0029A42F7D1AB
S32500000300FC22C4F20002136840F2FF319B059B0D8B4210D04EF20C034EF25451C4F2020340
S32500000320C1F6CC21196011684EF20402C4F20202116000221A60BDE8F00F704742F2EC2079
S3250000034008B5C0F2000000F011F94FF0FF3000F0FBF8002008BD00BF42F2A42008B5C0F2D2
S32500000360000000F003F9BDE80840FFF7E7BF00BF002070470020704700207047411C10B59C
S3250000038004460ED0C21C15D0831C07D000F07F44B4F17F4F02D06FF0100010BD6FF008005B
S325000003A010BD074800F0E2F8204600F003F96FF0280010BD034800F0D9F86FF0080010BD6B
S325000003C01C2300003423000008B500F01BF8FFF7C3FFBDE8084000F029B800BF08B5FFF7D9
S325000003E0C7FF002804DB00F0C5FF002800DB08BD034800F0BBF8BDE8084000F0A3B800BFC9
S325000004004C23000008B500F05DFE002804DBFFF7B1FF002800DB08BD034800F0A7F8BDE86B
S32500000420084000F08FB800BF6423000010B50446FFF7A2FF002C06DB054800F097F8BDE8CD
S32500000440104000F0E9B92046FFF798FFF7E700BF7C230000012910B419D016DD0378A3B1EC
S3250000046048F2050248F20804C4F20302C4F20304137803F00203DBB2002BF9D0034610F822
S32500000480011F21705B78002BF2D110BC704748F20502C4F20302137803F00203DBB2002B2A
S325000004A0F9D0027848F20803C4F203031A70ECE7012900D0704748F20502C4F2030213785D
S325000004C003F00403DBB2002BF9D048F20803C4F203031B78037070474FF45452C4F2030239
S325000004E0116843F2080321F0800170B4C4F203031160196843F21C6241F006011960C4F2BF
S325000005000302166848F201034FF4004546F040061660C4F203038020012248F20C04C4F21B
S325000005200305187048F204012A70C4F20304AC222280C4F20301002218700A7003221A7092
S3250000054070BC7047FEE700BF10B582B000F034F8012104460DF10700FFF7AAFF204600F095
S3250000056031F89DF8070002B010BD00BF38B5044600F022F8237805462BB914E0FFF76AFF14
S3250000058014F8013F7BB10A2B20464FF00101F5D10748FFF75FFF20460121FFF75BFF14F8B4
S325000005A0013F002BEFD1284600F00CF8002038BDE8220000FEE700BFEFF31180034981F3B2
S325000005C01188704780F31188704700001000000010B50446FFF7F0FF04F01F03012202FAC9
S325000005E003F36409A40004F1604404F561442360BDE81040FFF7E6BF10B50446FFF7DCFFC4
S3250000060004F01F03012202FA03F24EF280136409CEF2000343F82420BDE81040FFF7D2BFAC
S3250000062000F01F03012202FA03F34009800000F1604000F562400360704700BF00F01F03B1
S32500000640012202FA03F24EF280234009CEF2000343F82020704700BF00F01F03012202FA6F
S3250000066003F24EF280234009CEF2000353F8203013420CBF00200120704700BF70B50446AF
S325000006800D4616462D01FFF797FF04F00303DB0006F00F01FF22EDB20D4302FA03F205FA10
S325000006A003F324F0030404F1604404F56444216821EA020213432360BDE87040FFF782BFEC
S325000006C010B50C468047002800DB10BD2046FFF74DFF0348FFF74AFFBDE81040FFF732BF58
S325000006E09423000010B50446FFF766FF27482849FFF7E6FF27482849FFF7E2FF2748284981
S32500000700FFF7DEFF27482849FFF7DAFF27482849FFF7D6FF27482849FFF7D2FF274828491F
S32500000720FFF7CEFF27482849FFF7CAFF27482849FFF7C6FF27482849FFF7C2FF274828493F
S32500000740FFF7BEFF27482849FFF7BAFF27482849FFF7B6FF27482849FFF7B2FF274828495F
S32500000760FFF7AEFF204600F05DFA002808DB002100F0D4FA002803DBBDE8104000F00FBA85
S325000007802048FFF7F3FEFFF7DDFEF5E7010A0000B0230000E9090000B42300005D11000042
S325000007A0BC230000E10F0000C42300003D0E0000D02300007D0E0000DC230000390F00006D
S325000007C0E4230000A10F0000F4230000790F000000240000110F00000C240000BD0E00007E
S325000007E00824000021100000182400006510000028240000A9100000382400007908000003
S32500000800442400004C24000008B500F059F8BDE8084000F0F7B800BF08B5FFF7F5FFBDE865
S32500000820084000F0E3B800BFF0B4124E3168B14217D0D0E90245D1E90223A21A65EB0303B8
S32500000840002A73F1000709DA0BE0D1E90223A21A65EB0303002A73F1000702DB0968B14268
S32500000860F3D14B6880E80A004B6848601860F0BC704700BF40E1FF1F4EF2401110B5C1F648
S32500000880FF7100220023C1E90223C1E90423062409604960FFF790FE4EF210034EF2140294
S325000008A041F67F21CEF2000364F31F41CEF200021C60116007221A60FFF784FE002010BD2A
S325000008C04EF21003CEF2000300221A60704700BF43614B1C70B40261064604BF0060406049
S325000008E00FD0094BD3E90423521843EBE1730A240025121943EB0503C0E9022370BCFFF74C
S3250000090093BF70BC704700BF40E1FF1FF0B44EF24014C1F6FF7404F11005D5E900456418B3
S3250000092045F100050A260027A41945EB070502614361C0E90245F0BCFFF776BF10B4019CF7
S32500000940C0E902230461029C446110BCFFF76CBF2DE9F84300F031F9FFF72EFEDFF88490B6
S325000009600A24D9E904230025121943EB0503C9E90423804600260027D9E90445D9F80010FC
S32500000980494515D0D1E90223121B63EB0503964277EB03000CDB0B6899421FBF4A68136007
S325000009A00B685A600B69002BE8D048699847E3E7B8F1000F08D1084B1A68084B1B689A423B
S325000009C002D0074B1B6823B14046BDE8F843FFF7F9BD00F0EEF8F7E7A4F0FF1FA0F0FF1F70
S325000009E0A8F0FF1F40E1FF1F0020704708B5FFF7E3FD0020FFF7DEFDFFF7A4FDFCE700BF68
S32500000A0000207047704700BFDFF8C8D1DFF8C8C17248CCF80000724C724820607248DFF8AC
S32500000A20CCC1C0F800C000F015B84DF804ED6A486A490160DFF8B8E1DEF800E02DE9F04F77
S32500000A40674C6848D4F80080B8F1000F18BFC8F874D02060674D684E684880F31188D5F8DB
S32500000A600080B8F1000F40F00C80D6F800C0BCF1000F08BFFFF7C8FB5A4880F31188FFF70E
S32500000A80EBBFC4F80080D8F874D0534855490160BDE8F04F5649C1F800E05DF804EB5148C3
S32500000AA080F31188EFF31180704700BF00B5DFF850C1DCF8001001F10101CCF80010EFF310
S32500000AC00580A0F11000DFF83CC14FEA80015CF801C0E047DFF828C1DCF80020A2F10102D6
S32500000AE0CCF800205DF804EB704700BF704700BF454870471EF0040F0CBFEFF30881EFF35F
S32500000B0009818A6912F8021CDFF82400002908BF3E48102908BF3D483D4A904202BF3A4A96
S32500000B20009200F005B8069941F001010591069070472DE9FF5008ADDFF8B4C0DCF8007012
S32500000B404DF8047D6E464FEA074ECCF800E0D5F800C0BCF1000F80F20F8000F00AB8B546EC
S32500000B605DF804CB224CC4F800C004B0BDE8F05070472548FFF7F3BF296800F023F9FFF769
S32500000B80EEBF00BF2DE930501D4C256805F101002060FFF7DDFE2560BDE8305070471D4849
S32500000BA01D490860BFF34F8F4FF00000FFF70AFD70470D481949016070470B4818490160FA
S32500000BC07047EFF303807047EFF311807047EFF310807047001E0020A8F0FF1F01000000F4
S32500000BE0A4F0FF1F0000000004ED00E00000000838E1FF1FA0F0FF1F1C070020100000002C
S32500000C001807002058E1FF1FF6FFFFFF330B0000300B00002F00000000EF00E000000010BE
S32500000C200000000242682DE9F04B22F4487323F001030546002B65D1C368013B1F2B5CD838
S32500000C4003697F2B59DD03F10708920628F0070840D5434551D1C669FFF7AEFC2B4A8146B6
S32500000C601468944208BF6FF021041FD02368EF681360216868684A602968AA6820F4407320
S32500000C804FF0010C07F1FF3B06EB08072046E1602361626184F820B0C4F81880276784F838
S32500000CA01CC0A4F81EC000F0A1FAA468B9F1000F08D1174B1A68174B1B689A4202D0164BD7
S32500000CC01B68BBB14846FFF77DFC002C0BDB2046BDE8F08B404600F0E5FA06460028BBD135
S32500000CE06FF02004F3E76B689B06F0D4304600F00FFBECE7FFF75DFFE4E76FF01004204620
S32500000D00BDE8F08B6FF00A04E1E700BFB0F0FF1FA4F0FF1FA0F0FF1FA8F0FF1F244B70B551
S32500000D201B680E46002B23DD441E1F2C3CD8214BC4EB041403EBC404FFF73EFC94F82330F2
S32500000D400546082B25D0002B14BF6FF028046FF0290445B9184B1A68184B1B689A4202D08E
S32500000D60174B1B6893B12846FFF72CFC204670BD114B1B68002BD7D028B1441E1F2C13D803
S32500000D809B688342D3D16FF02804EFE7FFF711FFE9E7636FE26820469E62DA6200F058FAAA
S32500000DA00024002DDFD1D5E76FF01104DEE700BF18070020B8F0FF1FA4F0FF1FA0F0FF1F13
S32500000DC0A8F0FF1F70B5CBB2013B032B82B004462AD8174A1748126800EB8305002A06DD13
S32500000DE020462B6898470446204602B070BD124E3368002BF4D00191FFF7DEFB3368002080
S32500000E00DA8B0132DA83FFF7DDFB2B680199204698470446FFF7D0FB33680020DA8B013A31
S32500000E20DA83FFF7CFFBDFE76FF00904DCE700BF1807002020EDFF1FA4F0FF1F0D490E4A11
S32500000E4070B4A2F118030C46096002F5B476002542F8141C42F8105C42F8184C18460B6042
S32500000E6018331832B3420146F2D3024B5860002070BC704718E2FF1F38E2FF1F0D490E4AD0
S32500000E8070B4A2F11C030C46096002F1C406002542F8181C42F8145C42F81C4C18460B6056
S32500000EA01C331C32B3420146F2D3024B5860002070BC7047A0E3FF1FC4E3FF1F124A134B66
S32500000EC02DE9F001A2F138061F461B60194606F13008334606F5E07C00209D1B42F8300CA8
S32500000EE01C4648F8050042F8341C42F8387C0B603833383263452146EFD3044B00205C6091
S32500000F00BDE8F001704700BFC8E4FF1F88E4FF1F4EF25863C1F6FF734EF25062C1F6FF722D
S32500000F20194600209860D86341F8342F5A6013609B631960516070470D490E4A70B4A2F1EC
S32500000F4034030C46096002F5B676002542F8301C42F82C5C42F8344C18460B6034333432B9
S32500000F60B3420146F2D3024B5860002070BC7047C0E6FF1FFCE6FF1F4EF67003C1F6FF73BE
S32500000F804EF66802C1F6FF72194600209860986241F8202F5A6013605B62196051607047B1
S32500000FA00D490E4A70B4A2F124030C46096002F16C06002542F8201C42F81C5C42F8244C88
S32500000FC018460B6024332432B3420146F2D3024B5860002070BC7047B0E8FF1FDCE8FF1FF4
S32500000FE00D490E4A70B4A2F11C030C46096002F5D276002542F8181C42F8145C42F81C4C8E
S3250000100018460B601C331C32B3420146F2D3024B5860002070BC704748E9FF1F6CE9FF1F99
S325000010200E4B0F49A3F1300270B40C46096002F1C006002502F1300043F82C1C43F8285C11
S3250000104043F8304C3033B0420A60114601D20246F0E7034B00205A6070BC704748EBFF1F6F
S3250000106010EBFF1F0E4B0F49A3F1280270B40C46096002F5A076002500E0024602F128008E
S3250000108043F8241C43F8205C43F8284C2833B0420A601146F1D3034B00205A6070BC70478C
S325000010A008ECFF1FD8EBFF1F4EF6205340F6F122C1F6FF73C0F200021A605A609A60DA60F2
S325000010C00020704770B51848184900F0E1FE041E1EDB1749174A184B126052600846096064
S325000010E003F510750A460024A3F1480143F8442C43F8480C116003F8404C48330026AB425C
S325000011000A46F1D10A4B596000F0C4F9041E03DA00F016F8204670BD084B34461E6000F031
S325000011206FF9204670BD00BF80EFFF1F6824000030EDFF1F38EDFF1F88EDFF1F8CEFFF1F2C
S3250000114010B500F075F900F0DFF904464EF68070C1F6FF7000F0B8FE204610BD1D4A002397
S3250000116070B513601C4A1D4813602022026000EBC30101330A1D202B4A605260174CF6D114
S3250000118000263146042204F58470C4F80461C4F80C6100F0DBFD124A1249134B0E601546A9
S325000011A0304612601146421CA3F1780443F8741C43F8702C03F8556C43F8102C43F8785C98
S325000011C07833202A0C6010462146ECD1044B00205C6070BDA0F0FF1FA4F0FF1F90EFFF1FD9
S325000011E0B0F0FF1FA8F0FF1F30F1FF1F90F82410F0B4002390F82040026F456990F91C7097
S3250000120001F0FE0163F341014FF0080C0363436380F824108363C36680F823C080F82140F2
S3250000122080F82240C78325F0010542F8283C42F80C3CA2F148066FF006014FF0807342F896
S32500001240241C42F8043C42F8085C4667F0BC704770B5124E90F82250012280F8232006EBD2
S32500001260C5039A68043342605A68044603605C6006F584701460294600F0A4FD94F8243057
S3250000128003F00203DBB20BB1C6F80C4133689D42BFBF024B1D60024B1C6070BD90EFFF1FA7
S325000012A0A0F0FF1FF8B510240F28264603D9C61D26F007063446FFF77FF9144D2146074617
S325000012C0286800F043FA2B6804460C3398421BD000F088FAE3689B1B172B0AD854F8043C47
S325000012E043F0010344F8043C3846FFF76BF92046F8BDA619A4F10800314600F095FA286860
S32500001300314600F043FAE9E70024EDE71407002070B50546FFF750F9064615E9110024F002
S32500001320010445F8044C4268D20716D56368DB0748BFA5F1080406D404F1080000F052FA3E
S32500001340206800F07DFA0A4B2146186800F01EFA3046BDE87040FFF735B9083000F042FA41
S3250000136055F8080C00F06CFA55F8044CDEE700BF14070020F8B51F4BDFF880E01D68DEF8AB
S325000013800030B5F1202F2E4624BF4FF020263546073323F0070303F11404174F361B1A4651
S325000013A0A6F11001083E03F10C0C3B60A61942F8041B1046C3F80CC0C3F810C05A609A605E
S325000013C03146CEF8005000F02FFA38682146043000F02AFA72683B6842F0010272609A688C
S325000013E0184642F001029A60214600F0CFF90020F8BD00BF30E1FF1F1407002034E1FF1F0A
S3250000140010B54EF68074C1F6FF740021204600F025FD002240F20873C2F2000320461146C3
S325000014201B605B609A60BDE8104000F01BBD00BF70B5154D2B68002B24D00021134800F055
S325000014400DFD134BAA6819682C6800268A1AAC421A60AE6010D00021A6600C4800F002FD6D
S325000014600021A4F1080000F051F80021074800F0F5FC2C68AC42EED104480021BDE870401B
S3250000148000F0F0BC70BD00BF0807002080EFFF1F20070020F0B4184A184D0023164612605F
S325000014A0284611461F469C010133076162194030102B516066510A601146F4D1104A0E48FF
S325000014C0104D0023416016461260284611469C46342707FB03F40133C0F808C06219343089
S325000014E0102B516066510A601146F2D1044B00205A60F0BC704700BFB8FFFF1FC0FFFF1FC2
S32500001500C0030020C8030020002070472DE9F04F044683B08B468948002100F09FFC636934
S325000015204FF00009D3F838A0D3F834805F6900F093F9236B60634B45C4F8389040F3CB8014
S32500001540E36A7F4D0193FFF737F82B684846DA8B04F120060132DA83FFF734F8DDF804E0A7
S32500001560E16A226B3B465EF8040CD047FFF724F82B684846DA8B013ADA83FFF723F8A36B40
S325000015800133A36300216D4800F06CFCA36B002B05DDE06B01214FF0FF3200F0D5F9002106
S325000015A06163664800F05AFCD4F82090B1452ED0634D99F81C30002143F0100389F81C303C
S325000015C05E4800F04FFCFEF7F7FF2B680020DA8B0132DA83FEF7F6FF01214FF0FF323B4694
S325000015E009F11000C047FEF7E7FF2B680020DA8B013ADA83FEF7E6FF0021504800F02EFC9C
S32500001600484600F043FAD4F82090B145D1D100214A4800F027FC0021484800F01FFC6569A5
S32500001620484A48F63963C2EB0509C3F6E3034FEAE90903FB09F9A669E06BEF6AD5F814809F
S3250000164000F012F92046002100F002FA09F101092846314606EB092900F02CFA50B1AD69DD
S3250000166015F0010504D12946344800F0FBFB1FE02BF0010B3148002100F0F4FB3D46BFB121
S325000016802F4EFEF799FF33680020DA8B0132DA83FEF798FF424659464846B8470546FEF70A
S325000016A08BFF33680020DA8B013ADA83FEF78AFF0021224800F0D2FB234B00215A68236048
S325000016C062605A681D4814605C6000F0CBFB284603B0BDE8F08F264656F8205FB5423FF48D
S325000016E051AFDFF85C9003E02D68B5423FF44AAFEB68002BF8D02B7F43F010032B77FEF7B9
S325000017005BFFD9F800300020DA8B0132DA83FEF759FF05F1100101223B46E868D047FEF7FF
S325000017204BFFD9F800300020DA8B013ADA83FEF749FFA36B0133A363D6E700BF80EFFF1FAD
S32500001740A4F0FF1F40EDFF1FB8FFFF1F0268D31C32EA220228BF1A46B1EBA20F00F10C0384
S32500001760184609DD0022406883420CD0C2689142F9DB07DD006870470068834202D0C268B7
S325000017808A42F9DB70478A42F4DAFBE7F8B50D6801F10806AD1B0C4629460746FFF7D6FFAD
S325000017A063680C3723F00103B842636002D0C368AB4209D04368A060E360436846601E60C1
S325000017C0002365612361F8BD8268234643F8102F40F8083F2269606102B153600023A360BD
S325000017E0F8BD00BF036810B4BBB182686AB14368A2F1080142F8043C436842F8080C19609C
S32500001800C4688268036841605460984203D04268136003685A6010BC70478368C2681360F2
S325000018208368002BF6D1F6E7036848600B60036801605A6802F0010211435960704700BF64
S325000018404268036822F0010213600368596801F001010A435A607047024B186800B18068A2
S32500001860704700BFA4F0FF1F01380F28F8B52CD8C0EBC0008700FEF79FFE154E0546BC1912
S32500001880A36883B96FF0290445B9124B1A68124B1B689A4202D0114B1B689BB12846FEF776
S325000018A091FE2046F8BD204600F036F90C4B00225968BB5161600C605C60A2601446002D3B
S325000018C0ECD1E2E7FFF775F9E8E76FF01104E8E750E9FF1FA4F0FF1FA0F0FF1FA8F0FF1F99
S325000018E048E9FF1F70B5C66A144A013EC6EBC6060029034602EB860603DB3046194600F096
S325000019006BF933699B0717D43468B44214D07269E36B25689A4204DA0FE0E26B2D689A42A1
S325000019200ADC204600F0D6F8E26B7369AE42C2EB03032C467361F0D170BD70BD50E9FF1F13
S325000019404FF0FF31FFF7CEBF2DE9F043441E002383B00F2C01930D46914666D8994267DD38
S32500001960B2F1FF3F64DB344E3368002B3AD1334B1B68002B36DCDFF8D480D8F80030002B5A
S3250000198030D0FFF721F900282CD12D4BC4EBC40403EB8404FEF710FEA368074693B96FF0A1
S325000019A0290301933FB9274BD8F800201B689A4201D03368CBB13846FEF704FE019803B0FF
S325000019C0BDE8F083A3699D42C4BF6FF010030193E8DC23699A071ED563699D4208DC5D1B8A
S325000019E06561DFE76FF01800E9E7FFF7E2F8E2E7D8F800302269144912F0010FA1F10C02DB
S32500001A0018BF114601AA99629A63DD632046494600F0B0F8C6E72046D8F8001000F0FAF84D
S32500001A20D8F800308342E5D1D6E76FF01100C6E76FF01000C3E700BFA8F0FF1F180700207E
S32500001A4050E9FF1FA0F0FF1F0CE1FF1FA4F0FF1F036898421FBF4268136003685A60034610
S32500001A6053F8082F9A421FBFC3681A608268536031B1054B5A68036042605A6858601060FF
S32500001A8000230361704700BFB8FFFF1F036898421FBF4268136003685A60054B5A68036094
S32500001AA042605A685860002310608360704700BFC003002050F8403F834203D107E01B686B
S32500001AC0834204D09A698A42F9D1012070470020704700BF034653F8502F10B59A4218BFD5
S32500001AE0436D04461EBF1A60026D5360036898421FBF4268136003685A6090F82330022B00
S32500001B0006D0042380F82330A36B00221A6010BDFFF79EFBF8E700BFF8B504680546A0420D
S32500001B2027D004276FF0320604E0A36B2C681E60A5421ED0234653F8502F9A421FBF636D50
S32500001B401A60226D536023689C421FBF6268136023685A6094F82330022B18BF84F8237008
S32500001B60E3D12046FFF774FBA36B2C681E60A542E0D1F8BD38B5174D04462B686FF03100B5
S32500001B809A6B106001B938BDA2680846DA62216900F050F82369DB0714D5236828689C4275
S32500001BA090F8221003D106E01B689C4203D093F822208A42F8D95A68036042605A685860CC
S32500001BC0106038BD2B6862681C605A6062686360136038BDA4F0FF1F0B6810B499421FBF70
S32500001BE04A6813600B685A60036891F82240984203D106E01B68984203D093F82220A242C2
S32500001C00F8D95A680B604A605A685960116010BC704700BF0368984208D00269D20706D5AC
S32500001C2091F8220093F82220904200D20B461846704700BF70B50E4C0546236893F823203A
S32500001C40012A0CD0042A02D1062283F82320094A03F150002946BDE87040FEF739BE1846EB
S32500001C6000F00AF82368022283F82320EFE700BFA4F0FF1F191D0000F8B5254D0446D5F84C
S32500001C800C3190F82260984221D023689C421FBF6268136023685A6094F82430DA0744BF9F
S32500001CA06FF3000384F8243006D405EBC6035A6804339342164F0ED0164B1A68A24200D0AE
S32500001CC0F8BDD5F80C211249CAB11A60F8BD0023C5F80C31D9E707F58470314600F07EF8A0
S32500001CE03B689E42E8D107F584703146C6F1200200F082F8002807DB30183860DCE70A68D9
S32500001D0001EBC2025268E0E720233B60D4E700BF90EFFF1FA0F0FF1F036810B5984218BF08
S32500001D20426804461EBF136003685A6090F82330022B08D0042380F82330A36A9B680BB196
S32500001D402046984710BDFFF783FAF6E7072A70B4C9B225D9860703462BD003F8011B013A2A
S32500001D609E07FAD10E0446EA01260E43032A46EA01660DD91D461446043C032C45F8046BB1
S32500001D80FAD8141F24F0030404341B1902F0030222B19A1803F8011B9342FBD170BC70479A
S32500001DA0002AFBD08218034603F8011B9342FBD1F4E70E0446EA01260E4346EA0166034618
S32500001DC0D8E700BF002908DB01F00703012202FA03F3C910425C134343547047002909DB3B
S32500001DE001F00703012202FA03F3C910425C22EA03034354704700BFCB0FF0B453EAD27733
S32500001E0025D101F00705012404FA05F4CE108119E4B2E2B1835DF3B91846C5F1080590B11E
S32500001E200830904213DA11F8013F002BF7D0234204D16400E4B201302342FAD08242D8BF7B
S32500001E404FF0FF3005E0284601249042EBDB4FF0FF30F0BC70473846E9E700BF4FF0FF32B0
S32500001E6000F042B838B5012505FA01F50446FEF7A3FB236823EA05032360FEF7A3FB60680F
S32500001E8000B938BDA0682946BDE8384000F0E2B870B5054686B099B101AE3046042200F045
S32500001EA0DDF90024092330460293039400F04AF8A042A860A2BF6C602C60204606B070BD36
S32500001EC006AE46F8141DECE710B504468068002806DD00F081F8002804DB0020A06010BDA7
S32500001EE06FF0100010BD00BFF0B5044685B00125174605FA01F5FEF75FFB63680133636034
S32500001F00FEF760FB05E0A068009700F011F9061E0EDBFEF751FB236845EA030105EA0306E9
S32500001F202160FEF74FFB2946212203AB002EEAD1FEF742FB6368013B6360FEF743FB3046ED
S32500001F4005B0F0BDF0B5436883B033F00902044634D1FEF731FB1B4A1368934208BF6FF01D
S32500001F60210417D018494AF6AB25591ACAF6AA25C9101E6805FB01F11660276866681D6833
S32500001F80A46801316A601B605C615B609960DF601E610C4640B90D4B1A680D4B1B689A42AD
S32500001FA002D00C4B1B6823B1FEF70CFB204603B0F0BD0190FEF7FDFD0198F5E76FF00A0477
S32500001FC0F4E700BF18E2FF1F20E2FF1FA4F0FF1FA0F0FF1FA8F0FF1F01380F28F8B52CD8F2
S32500001FE000EB4000C700FEF7E7FA154E0546BC19A36883B96FF0290445B9124B1A68124B83
S325000020001B689A4202D0114B1B689BB12846FEF7D9FA2046F8BD2046FFF77EFD0C4B0022BD
S325000020205968BB5161600C605C60A2601446002DECD1E2E7FEF7BDFDE8E76FF01104E8E714
S3250000204020E2FF1FA4F0FF1FA0F0FF1FA8F0FF1F18E2FF1F01380F282DE9F0410F464ED8FA
S3250000206000EB4000C600FEF7A7FA264C80463519AB6833B36B6930593B4385426B610DD009
S32500002080066CC46BF20707686B691DD51C420CBF00220122FAB938468542F1D10024B8F176
S325000020A0000F08D1184B1A68184B1B689A4202D0174B1B6803B34046FEF784FA2046BDE81A
S325000020C0F0816FF02904EAE704EA0302A11A4A424A41002ADFD0426C1360FFF7FBFCB206C8
S325000020E005D56B6923EA04046C61002CD6D0F306D1D500246C61D2E7FEF75BFDDBE76FF0C1
S325000021001104DBE720E2FF1FA4F0FF1FA0F0FF1FA8F0FF1F0146C06A4EF220230138C1F6C8
S32500002120FF7300EB400003EBC000FFF755BD00BF2DE9F047441E82B000200F2C01900E4666
S3250000214015469A467BD8002973D032F0310370D10A9B01336DDB3B4F3B68002B37D13A4BE2
S325000021601B68002B33DCDFF8F090D9F80030002B2DD0FEF729FD002829D1344B04EB440429
S3250000218003EBC404FEF718FAA3688046ABB96FF029030193B8F1000F08D12D4BD9F800202E
S325000021A01B689A4202D03B68002B45D04046FEF709FA019802B0BDE8F0872369180709D498
S325000021C02268944206D06FF028030193E2E76FF01800EFE7E907626910D516420CBF0021AB
S325000021E0012189B1CAF80020AA0642BF6369B3436361EB06CED500236361CBE706EA020144
S32500002200701A41424141ECE71249D9F8002013F0010FA1F10C0018BF014601AB91629363A6
S32500002220D6631564C2F844A020460A99FFF7A2FCB0E76FF01000BDE7FEF7BBFCB6E76FF059
S325000022401100B7E7A8F0FF1F1807002020E2FF1FA0F0FF1F24E1FF1FA4F0FF1F70B40446C3
S325000022601618013AB4420ED00D78234603F8015B11F8015B1C46002DF3D122B19A1803F89E
S32500002280015B9342FBD170BC704700BF08B5FEF7A5F842F2C820C0F20000FEF723FA00204A
S325000022A008BD00BF0A6D6963726F20542D4B65726E656C2056657273696F6E20312E303188
S325000022C02E30310A0A0000000000000001000000C90300001E00000000040000696E6974B2
S325000022E074736B00000000000D0000005075736820616E79206B657920746F207368757421
S32500002300646F776E20746865206D6963726F20542D4B65726E656C2E0A0000000A3C3C2088
S3250000232053595354454D2052455354415254203E3E0A00000A3C3C2053595354454D2052CE
S3250000234045424F4F54203E3E0A000000214552524F522120696E69745F6B65726E656C0ACE
S3250000236000000000214552524F52212073746172745F73797374656D0A0000000A3C3C208D
S3250000238053595354454D2053485554444F574E203E3E0A00203A206D6F64756C6520696E19
S325000023A0697469616C697A65206572726F720A0063707500746B6465760000007461736B4F
S325000023C00000000073656D6170686F72650000006576656E74666C61670000006D61696CD4
S325000023E0626F78006D65737361676562756666657200000072656E64657A766F75730000DA
S325000024006D757465780000006669785F6D656D6F7279706F6F6C00006379636C696368614A
S325000024206E646C6572000000616C61726D68616E646C657200000000737562737973746514
S325000024406D00000074696D6572000000696E69745F7461736B2063616E206E6F7420737458
S3150000246061727465640A0000444D4C6B0000000004
S3250000247004000000E51800004119000004000000000000004119000008000000152100004F
S31500002490000000000800000000000000000000002E
S70500000100F9
